:020000000628D0
:080008000B110900831685109D
:1000100083120130A200C32063200130A200C3205C
:100020000130003C031934282030A4008030240221
:10003000013003180001003C031933282408910003
:100040004320203091004320240893006A20203070
:10005000910043202408950097200130A200C3207E
:100060006320A40A162810280E0890006E308F0016
:100070000000000000000000000000008F0B382886
:10008000900B362808008510FF3092001208003CC3
:100090000130031900019203003C0319502846283F
:1000A0000930031003188510031C85145728103ECF
:1000B000031C5628FF3E910C031D522885100A3060
:1000C0008E0034200800FE30910043200130910062
:1000D00043200800003094001308633C01300318EB
:1000E0000001003C03197A286430130293001408BD
:1000F000940A6C283030140791004320003094009B
:100100001308093C013003180001003C03198E2834
:100110000A30130293001408940A80283030140720
:100120009100432030301307910043200800150848
:10013000F0399600960E0A301602013003180001BD
:10014000003C0319A8283030160791004320AD2841
:100150000A301602413E9100432015080F399600DF
:100160000A301602013003180001003C0319BD28B3
:100170003030160791004320C2280A301602413E53
:100180009100432008000030A3000A302302013010
:1001900003180001003C0319D22864308E0034207B
:0601A000A30AC5280800B7
:00000001FF
